:10F800000C94387C0C94537C0C94537C0C94537C57
:10F810000C94537C0C94537C0C94537C0C94537C2C
:10F820000C94537C0C94537C0C94537C0C94537C1C
:10F830000C94537C0C94537C0C94537C0C94537C0C
:10F840000C94537C0C94537C0C94537C0C94537CFC
:10F850000C94537C0C94537C0C94537C0C94537CEC
:10F860000C94537C0C94537C0C94537C0C94537CDC
:10F8700011241FBECFEFD0E1DEBFCDBF11E0A0E06D
:10F88000B1E0E2E2FFEF02C005900D92A030B107B7
:10F89000D9F712E0A0E0B1E001C01D92A434B10795
:10F8A000E1F70C94537F0C94007C0F92AF93BF93BD
:10F8B000CF93DF93EF93FF93FC01EA01DB01C8953F
:10F8C000099231961197D9F7FF91EF91DF91CF917E
:10F8D000BF91AF910F9008950F921F920F93AF9326
:10F8E000BF93CF93DF93EF93FF93FC01EA01DB011A
:10F8F0000990199001E043D032961297C9F7FC01A4
:10F9000003E03DD005E03BD0FF91EF91DF91CF9137
:10F91000BF91AF910F911F900F9008950F931F9378
:10F92000EF93FF93FC0103E02AD000E011E0E00F29
:10F93000F11FE617F707B9F7FF91EF911F910F91AC
:10F9400008950F930F9222D0082E09E018D00F903F
:10F950000F9108950F930F92EF93FF9317D0FC012F
:10F9600060935700C895802DFF91EF910F900F91F4
:10F9700008950F930BD001E102D00F910895F999EA
:10F98000FECF00935700E895FFFF0000009157005D
:10F9900000FDFCCF089589E08093C4008091C100F0
:10F9A00088618093C10008958091C100877E809313
:10F9B000C10008958093C6008091C00086FFFCCFEF
:10F9C0008091C00080648093C00008958091C6003B
:10F9D000992708958091C0009927807890700895A4
:10F9E000EF92FF920F931F93CF93DF937B01C0E0C1
:10F9F000D0E0C617D70770F48C010E94EA7C8823F8
:10FA0000E1F30E94E67CF80181938F012196CE15E7
:10FA1000DF0598F381E090E0DF91CF911F910F9186
:10FA2000FF90EF900895EF92FF920F931F93CF9363
:10FA3000DF937C018B01C0E0D0E0C017D10738F420
:10FA4000F70181917F010E94DA7C2196F6CF81E057
:10FA500090E0DF91CF911F910F91FF90EF9008956B
:10FA600040E050E04817590750F429EC38E0000016
:10FA70002150304037FFFBCF4F5F5F4FF3CF0895EA
:10FA80000E94D47C0E94000008950E94EA7C882392
:10FA9000E1F30E94E67C803219F481E090E0089561
:10FAA00085E10E94DA7C80E090E0089590E0282FC4
:10FAB00033272138310589F02238310524F42038E4
:10FAC000310549F00DC02238310549F0283931059A
:10FAD00039F493E005C092E003C091E001C092E1E7
:10FAE000892F9927089540E050E06091400170917E
:10FAF000410146175707D0F420914202309143024A
:10FB0000E2E4F1E032BD21BD2F5F3F4F808180BD37
:10FB1000FA9AF99AF999FECF4F5F5F4F31964617DF
:10FB2000570780F33093430220934202089540E048
:10FB300050E0609140017091410146175707B0F4C1
:10FB40002091420230914302E2E4F1E032BD21BD56
:10FB50002F5F3F4FF89A80B581934F5F5F4F4617F5
:10FB60005707A0F330934302209342020895CF93A6
:10FB7000DF93C0E0D0E08091400190914101C8172F
:10FB8000D907A0F4CE018E5B9E4F209142023091A6
:10FB90004302220F331FAC0160E071E0C9018C0FFA
:10FBA0009D1F0E946C7CC050DF4FE5CF0E94B97C46
:10FBB000DF91CF910895809142029091430242E4F7
:10FBC00051E06091400170914101880F991F0E949E
:10FBD000557C0895CF93C0E069E081E090E00E94F9
:10FBE000AA7C992784FF03C08F7E0E94A17C0E947B
:10FBF000EA7C8823E1F30E94E67C9927823591050F
:10FC00001CF5803591050CF05CC08134910509F438
:10FC100062C0823491057CF481339105B1F1823365
:10FC2000910524F4C09709F44CC037C18034910584
:10FC300009F437C132C18234910509F45FC08534BB
:10FC4000910509F45EC029C18635910509F4F0C01B
:10FC5000873591054CF48235910509F45FC08535EF
:10FC6000910509F468C019C18437910509F4A3C04E
:10FC7000853791052CF48436910509F475C00DC1C2
:10FC80008537910509F4C4C008C10E94457D8823C9
:10FC900009F4ADCF84E10E94DA7C81E40E94DA7C31
:10FCA00086E50E94DA7C82E50E94DA7C80E20E948E
:10FCB000DA7C83E50E94DA7C84E50E94DA7C8BE4BE
:10FCC00006C00E94457D882309F491CF84E10E94FB
:10FCD000DA7C80E1E3C061E070E080E091E00E94C6
:10FCE000F07C0E94457D882309F481CF84E10E9445
:10FCF000DA7C809100010E94567DE9CF64E170E0DA
:10FD000008C061E070E080E091E00E94F07C64E077
:10FD100070E080E091E00E94F07CD3CF0E94457DAE
:10FD2000882309F464CF60E070E0CB010E948E7CF0
:10FD30000E94B97CCBCF62E070E080E091E00E944D
:10FD4000F07C0E94457D882309F451CF2091000169
:10FD5000809101019927982F8827820F911D9093F8
:10FD6000430280934202B2CF63E070E080E091E012
:10FD70000E94F07C20910101809100019927982F29
:10FD80008827820F911D9093410180934001BC010F
:10FD900082E491E00E94F07C0E94457D882309F472
:10FDA00026CF80910201863419F40E94B77D8ECF50
:10FDB0000E94737D8BCF63E070E080E091E00E9451
:10FDC000F07C20910101809100019927982F8827CC
:10FDD000820F911D90934101809340010E94457DC7
:10FDE000882309F404CF80910201863419F40E941B
:10FDF000DB7D02C00E94977D84E10E94DA7C6091E5
:10FE000040017091410182E491E00E94137D61CF35
:10FE10000E94457D882309F4EACE84E10E94DA7CC1
:10FE20008EE10E94DA7C86E90E94DA7C89E04FCF7D
:10FE300064E070E080E091E00E94F07C0E94457DEB
:10FE4000882309F4D4CE84E10E94DA7C80910001F9
:10FE5000803531F480910101882361F4C82F17C0E7
:10FE6000883531F480910101883061F4C3E00FC01E
:10FE7000803531F480910101883049F4C2E007C037
:10FE8000883529F480910101882309F4C1E069E0F3
:10FE90008C2F99270E94AA7C1ACF85E10E94DA7CD8
:10FEA000A6CECF910895CFEFD0E1DEBFCDBFCEE19A
:10FEB000F894AEEFB7E00E94887F802D843B79F400
:10FEC000AFEFB7E00E94887F802D833C41F4ADEF17
:10FED000B7E00E94887F802D9927809366000E945A
:10FEE000CB7C0E94E67C84E690E00E94307D0E94FC
:10FEF000EA7C882319F00E94EA7D04C0C150C5B98C
:10FF0000CC2389F70E94407D80E090E00C94907FA4
:10FF1000F999FECFB2BDA1BDF89A119600B408952B
:02FF2000FFCF11
:040000030000F80001
:00000001FF
